:1000000009C016C015C014C013C012C011C010C062
:100010000FC00EC011241FBECFE9CDBF10E0A0E677
:10002000B0E001C01D92A338B107E1F748D0D4C0B9
:10003000E7CF8FEE87BB08951F9352E010E080E07A
:1000400090E025E530E066B3462F407164FD0DC0B9
:10005000552359F0123248F4E12FF0E0E05AFF4FF7
:10006000B901A6D060831F5F25C001965BE0893B84
:10007000950710F11F31C8F0E3E6F0E083E090E06F
:1000800020E030E0A901612F70E008C0A191A1112A
:100090002160220F331F441F551F019686179707B3
:1000A000ACF3B901CA011F9108955CE08D31950749
:1000B00018F010E080E090E000C0542FC4CFCF9241
:1000C000DF92EF92FF920F931F938FEB94EDA1E0DD
:1000D00081509040A040E1F700C000008FEE87BB48
:1000E00018BAA7E9BAE31197F1F700C000000AE0D7
:1000F000C02E14E0D12EB9E0EB2EFF24F39406E0DD
:1001000015E09ADF6A3FB4E07B07B5E98B07BAE6F2
:100110009B07E1F16B3F24E0720725E982072AE69D
:100120009207CCF46A37A5E87A07A4E98A07AAE619
:100130009A0781F16E35B1EA7B07B4E98B07BAE61D
:100140009B0751F16A3F25E0720724E982072AE6FE
:10015000920739F519C06A37A4E87A07A5E98A0732
:10016000AAE69A07A9F06E35B0EA7B07B5E98B07D6
:10017000BAE69B0799F06E3C20E3720725E98207F7
:100180002AE6920771F40CC018BB0BC0C8BA09C0AC
:10019000D8BA07C0F8BA05C008BB03C0E8BA01C0A6
:1001A00018BA8BED95E00197F1F700C00000A9CFD8
:1001B000AA1BBB1B51E107C0AA1FBB1FA617B7078D
:1001C00010F0A61BB70B881F991F5A95A9F78095A9
:0C01D0009095BC01CD010895F894FFCF7C
:00000001FF
